:020000040000FA
:060000008A0183017D2846
:08000800A000030EA100A219E3
:100010000C28000085100E2885140E28A2108519C2
:100020001628221C1428A21422101A2822140000B8
:1000300000001A28A411051822280000241AA4156B
:1000400024122628241EA415241626282217221A34
:100050003128A21C3F280230AB000A30AA00221629
:100060003E28AB0B3E280430AB00AA0B3A282212E4
:1000700022153E280314221C0310AC0CA210231BD3
:100080004B28241D5C282708A5000A30A60024114F
:10009000231703105528231F5C28A80B5C28A60BE8
:1000A000532823135C280314A50CA2110318A215CE
:1000B0000430A8005C28A313A4196F282E302D0645
:1000C00003197728AD0A2D302D06031D7728A216B7
:1000D000241EA2122D08AE002314A4167728A216FF
:1000E000241AA21223142D08AE00AD0177280B119B
:1000F000210E8300A00E200E090085018510073017
:10010000990083168F308100990100309F00F930EB
:1001100085008C01831200309F008312A201A3018D
:10012000A401A2158514051598220511982205151C
:100130009822051198220515982205119822051577
:100140009822051198220515982205119822B101CF
:10015000B401AD014130B200B30083168C019601A9
:1001600083128C018B018B168B170130D8003B2139
:10017000640021212219C928A3181529A418C3280D
:10018000A41BC62815295E21A41015297F21A413BC
:1001900015292211A318D32802302C06031D152976
:1001A000A314B50115292319D9282C08D800231523
:1001B0001529A319EE282C08D9000F39023EDC00BE
:1001C000A31558080F39013A0319152902309A214D
:1001D00058089A2159089A21A3161529A31A092902
:1001E000231AF7282C08DA002316DC0315295D08EA
:1001F000DB002C08DD00DC0B152901305A06031D3D
:10020000032924210D2902305A06031D0D293B2103
:100210000D29DC0B13292C089A21A3102311A311FB
:100220002312A31215292C089A21B82846309A21A6
:1002300036309A2146309A2142309A2142309A2112
:100240000800BA21A7210800B50102309A21580EF2
:10025000B5079A210F30D905340E5904B5079A21F4
:1002600092225A08B5079A215B08B5079A21B50969
:10027000350A9A210800B50102309A21580EB507B7
:100280009A210530D900340E5904B5079A219222DB
:100290000230B5079A215230B5079A215830B50778
:1002A0009A212030B5079A215630B5079A2132306D
:1002B000B5079A21B509350A9A210800B50102301F
:1002C0009A211030B5079A21340E0538B5079A21C6
:1002D00092223608B5079A213708B5079A213808BF
:1002E000B5079A213908B5079A213A08B5079A2126
:1002F0003B08B5079A21B509350A9A210800B501CE
:1003000002309A211030B5079A21B103340E31041E
:10031000B5079A219222B10ADF0136305F078400C7
:100320000008B5079A21DF0AB10B8D29B509350AF6
:100330009A210800DE00320884005E088000B20ABC
:1003400058303206031D08004130B2000800320860
:100350003306031908002419080033088400000834
:10036000A7002415B30A58303306031D0800413096
:10037000B3000800231C2A2AA4182A2AA41B2A2A0C
:100380002310A21BD829241CC829241B2C2AE829A5
:10039000A21E2A2A0C30AE02031CF7291230AE022C
:1003A0000318F729B1010830AF002414A217FA2965
:1003B000A21324170530AE02031CF7290730AE0242
:1003C000031C2A2A0C30AE020318F72924132A2A08
:1003D000A21EFD29EB290630AE02031CF7290930C5
:1003E000AE02031CF8290F30AE02031CFA29242A9E
:1003F0000314FB290310B00D0B2AA41A082A0D3090
:10040000AE02031CF7291030AE02031C2A2AF7297A
:100410002410B00E0F2AAF0B2A2A0830AF00310883
:10042000031D172A0A303006031D242A051536300D
:100430003107840030088000310A063A0319272A60
:10044000063AB100B0012A2A241005112A2AA41460
:1004500024100511A4120800A21E4D2A2F2A0530CF
:10046000AE02031C3B2A0630AE02031C3C2A0830B5
:10047000AE02031C3E2A8A2A03143F2A0310B00D41
:10048000902A0530AE02031C3B2A0630AE02031C44
:100490003C2A0830AE02031C3E2AA41A612A053009
:1004A000AE02031C3B2A0630AE02031C5E2A083053
:1004B000AE0203183B2A301C3B2A712A30183B2A13
:1004C000712A2410310803198A2A682A0310B00DF2
:1004D000AF0B662A36303107840030088000B10A3D
:1004E0008D2AAF0B902A0830AF003108031D7D2AFA
:1004F00000303006031D8A2A051536303107840086
:1005000030088000310A0B3A03198D2A0B3AB100EA
:10051000B001902A24100511902AA4172410051167
:10052000A4120800B40A3408103A0319B40E0800E3
:10053000F030DF00DE01640000000000DE0BA12AC5
:06054000DF0B9B2A0800FE
:02400E00CA3FA7
:00000001FF
